:04000000FDEF07F019
:100F000055415254313A20284552524F5229206FB0
:100F100076657272756E0D0A0000016E010E010198
:100F20000101006F0150016E010E02010201006F0C
:100F30000150016E010E03010301006F0150016EAB
:100F4000010E04010401006F0150016E010E050144
:100F50000501006F0150016E010E06010601006FD0
:100F60000150016E010E07010701006F0150016E73
:100F7000010E08010801006F0150016E010E090108
:100F80000901006F0150016E010E0A010A01006F94
:100F90000150016E010E0B010B01006F0150016E3B
:100FA000010E0C010C01006F0150016E010E0001D9
:100FB0000001606F0150016E010E0D010D01006F07
:100FC0000150016E010E026E0150016E010E000112
:100FD0000001C46F0150016E010E0D010D01646F1F
:100FE0000150016E010E346E0150016E010E0D01B3
:100FF0000D01966F015000EF00F00DEEAAF011EE1A
:1010000000F0EE6AE550E150FCE1E250FAE12C0E0E
:10101000F66E100EF76E000EF86E0900F5CF5CF05C
:0E1020000900F5CF5DF000018DEF07F0AA0D7D
:020000040001F9
:08FFF8008AF48DF0A7F87FF3F5
:00000001FF
